:020000040000FA
:0400000004EF00F019
:08000800F4EC00F0F3EC00F051
:10001000F2EC00F0926A936A946A016A026A0250F2
:1000200001260152D8A417EF00F0010E026E015014
:100030001508D8A41EEF00F0FF0E026E8A90015240
:10004000D8A48A80EBEC00F08A9201500108D8A471
:100050008A82EAEC00F08A9401500208D8A48A84CB
:10006000E9EC00F08A9601500308D8A48A86E8ECEF
:1000700000F08A9801500408D8A48A88E7EC00F0C0
:100080008A9A01500508D8A48A8AE6EC00F08A9C76
:1000900001500608D8A48A8CE5EC00F08A9E015035
:1000A0000708D8A48A8EE4EC00F08B900150080871
:1000B000D8A48B80E3EC00F08B9201500908D8A4FF
:1000C0008B82E2EC00F08B9401500A08D8A48B8458
:1000D000E1EC00F08B9601500B08D8A48B86E0EC85
:1000E00000F08B9801500C08D8A48B88DFEC00F04E
:1000F0008B9A01500D08D8A48B8ADEEC00F08B9C03
:1001000001500E08D8A48B8CDDEC00F08B9E0150C2
:100110000F08D8A48B8EDCEC00F0899001501008F9
:10012000D8A48980F1EC00F0899201501108D8A47C
:100130008982F0EC00F0899401501208D8A48984D7
:10014000EFEC00F0899601501308D8A48986EEECF4
:1001500000F0899801501408D8A48988EDEC00F0CB
:10016000899A01501508D8A4898AECEC00F0640E35
:10017000BEEC00F00FEF00F0BCEF00F0036E035098
:10018000046E0A0E056E010EC6EF00F0066EFF0E3D
:10019000076E0550096E0450086EEF0E0724D8B0A4
:1001A000CEEF00F0082ECDEF00F0092ECBEF00F0DF
:1001B000062EC9EF00F01200120012001200120009
:1001C000120012001200120012001200120012009F
:1001D000120012001200120012001200120012008F
:0E01E0001200120012001200060EC16E120074
:0200000400F00A
:020000040030CA
:0E00000000260E0E00008000F0C00FE00F4042
:00000001FF
